:100000000C9422040C948E040C94FE070C948E0421
:100010000C94AA090C948E040C948E040C948E04F7
:100020000C948E040C948E040C948E040C94171F64
:100030000C948E040C947F2D0C948E040C948E04DE
:100040000C948E040C948E040C948E040C94D42D79
:100050000C948E040C948E040C948E040C948E04D8
:100060000C948E040C948E040C948E040C948E04C8
:100070000C948E04310D3F0D4B0D4B0D230D4B0D8C
:100080004B0D4B0D4B0D4B0D4B0D4B0D4B0D4B0DB0
:100090004B0D4B0D4B0D4B0D250D4B0D270D4B0DEA
:1000A0004B0D4B0D4B0D430D4B0D5A0D410D4B0D93
:1000B0004B0D4B0D4B0D4B0D4B0D4B0D4B0D4B0D80
:1000C0004B0D4B0D4B0D4B0D1B0D370D290D3B0DE6
:1000D0004B0D2B0D4B0D2F0D4B0D390D2D0D3D0DDA
:1000E000330D350D4B0D4B0D4B0D4B0D4B0D4B0D7E
:1000F0004B0D1D0D1F0D210D450D470D4B0D4B0DCE
:100100004B0D490DF70DF90D030E030E030E030EF3
:10011000030E030EFB0DFD0DBF0D030E030EF90DB7
:10012000060E030E030EBF0DF70D030E030EFD0D9D
:10013000030E030E030E030E030E030EC10DF70D87
:10014000E30D030EE70D030E030E030EC30DFB0DAF
:10015000030E030EF10D030E030E030EC50D010E6B
:10016000030EE50D030EF90D030E030EF50DE90D5B
:10017000030EEB0DFD0D030E030E030EF30DED0D3F
:10018000030E030E030E030E030E030E030EEF0DFC
:10019000030EC70D030E030EFB0D030E030E010E1F
:1001A000030E030E030E030E030E030E030E030EC7
:1001B000030EC90D030E030E030EF10D030E030E05
:1001C000030E030E030E030E030E030E030E030EA7
:1001D000CB0D030ECD0DCF0D030E030E030ED10D6F
:1001E000D30DD50D030ED70DD90D030E030E030E3F
:1001F000FF0DDB0D030EDF0DDD0DE10D030E030E14
:10020000030E030E010EA50EF30ED20E190F3D0FB5
:10021000450F4C0F510F550F5C0F690F88108A1056
:100220008C108E10901098109810981092109410B6
:1002300096106C1184119811B311C511D011F411DD
:100240000D12331255123A13DF14DC16C1167D1D40
:10025000A41D9C1EA41D9C1EF01D131E9C1E6A1E28
:10026000791E5C235C23942394230F2443243A2691
:100270003A265A243A26EB23EB23F4253A2609267C
:100280002726722530325820005220006973723AB6
:100290002530345820007725303258200021435330
:1002A000335F4630210A00214353335F52454144B6
:1002B00059210A00214353335F5245534554210AC3
:1002C00000214353325F45305F4630210A0021430D
:1002D00053325F46302120253032580A00214353E3
:1002E000325F4530210A00214353325F494E495461
:1002F000210A00214353315F45305F2530325821B8
:100300000A00452575200050257520004D5B783A80
:10031000256420793A256420763A256420683A25B8
:100320006420623A253032585D0A000A5B434C5221
:100330005D20004C257520000A4D6F7573653A20CD
:1003400025730A000A4445463A20000A4558503AA7
:1003500020000A494E543A20000A4C4F473A2000E8
:100360000A4C4D533A200053257520000A49443A5F
:100370002530345828257325732920000A556E6BC3
:100380006E6F776E2049443A205265706F72742008
:10039000746F20544D4B20004E4720004F4B2000DF
:1003A0004E4720004F4B20000A353537365F435308
:1003B0003832683A005225752000572575200057BD
:1003C00025752000572575200058257520004125EA
:1003D00075200049257520005B4348475D20000AD1
:1003E0002575205052543A25303258204953523AFC
:1003F0002530345820000A2575204552523A2530C0
:100400003258204953523A253034582000535B2546
:10041000303258202530325820253032585D2000A7
:10042000007B46010203763A687F6577482B353BAF
:100430006978796439141E3C6A7A1D16041A1F3DC6
:100440006B061B070821203E6C2C19091715223F4B
:100450006D11050B0A1C23406E7E100D18242541DA
:100460006F360E0C122726427037380F33132D4388
:10047000717534322F2E44727C7D2830317445736F
:1004800051504A524D492A5466594F5C5F4C4B4E6D
:1004900062635A5D5E60295367585B5657614755E2
:1004A0004842403E3C3A3B456843413F3D2B357E08
:1004B000697A790078141E7B6A7C1D16041A1F7FE6
:1004C0006B061B07082120656C2C19091715224A99
:1004D0006D11050B0A1C234C6E49100D1824255173
:1004E0006F360E0C1227264F7037380F33132D52EC
:1004F000717534502F2E4E72397D28304D314B732B
:100500005464586776012A773259745C5F66020337
:1005100062635A5D5E60295344575B565561474696
:1005200080291E1F20212223242526272D2E2A2B19
:10053000141A0815171C180C12132F3028780416DB
:1005400007090A0B0D0E0F33343579311D1B0619BF
:100550000511103637387D557A2C393A3B3C3D3EF3
:100560003F4041424353475F6061565C5D5E57596F
:100570005A5B62634648644445677B7F65030102BA
:100580005250514F68696A6B6C6D6E6F7071725822
:1005900000494C754A4D734B4E767C777E74665499
:1005A0000A4C6F6F702073746172742E0A000A55C2
:1005B000534220636F6E666967757265642E0A0028
:1005C0000A544D4B3A6332303561352F4C55464114
:1005D0003A6436613764660A003403490042004DCC
:1005E0000020005000430020006B0065007900628D
:1005F000006F00610072006400200063006F006EF5
:10060000007600650072007400650072000000084A
:100610000354004D004B0000000403090409025478
:1006200000030100A03209040000010301010009D8
:100630002111010001223900070581032000010971
:100640000401000103010200092111010001227FC0
:1006500000070582030800010904020001030000ED
:100660000009211101000122220007058303200057
:10067000011201100100000008EDFEEE1B01020155
:100680000200010631FF0974A1010975150026FF5A
:10069000009520750881020976150026FF00952037
:1006A00075089102C005010902A1010901A1008597
:1006B0000105091901290815002501950875018111
:1006C000020501093009311581257F9502750881E0
:1006D0000609381581257F950175088106050C0AE4
:1006E00038021581257F950175088106C0C0050176
:1006F0000980A10185021601002637001A81002A0F
:10070000B700751095018100C0050C0901A1018594
:1007100003160100269C021A01002A9C02751095FE
:10072000018100C005010906A101050719E029E7BB
:100730001500250195087501810205081901290593
:100740009505750191029501750391010507190041
:1007500029F71500250195F875018102C0636F6EB8
:1007600073756D65723A20253034580A00737973B9
:1007700074656D3A20253034580A000A002530325D
:100780005820006B6579626F6172643A20004C45B5
:10079000443A20253032580A0025583A253031365F
:1007A0006225730A000A202030313233343536375F
:1007B00038394142434445460A0064656C5F6B65C5
:1007C000795F6269743A2063616E27742064656C96
:1007D0003A20253032580A006164645F6B65795FA6
:1007E0006269743A2063616E2774206164643A2000
:1007F000253032580A00290A002575002F0025757A
:10080000005D280025640020002564002000256488
:100810000020002564007C0025303258006D6F7583
:1008200073656B6579205B62746E7C7820792076C5
:1008300020685D287265702F61636C293A205B0027
:10084000560B6B1711241FBECFEFD4E0DEBFCDBF18
:1008500004B603FE41C08091220490912304A0912C
:100860002404B09125048730904BA740B04BA1F5EC
:100870001092220410922304109224041092250452
:1008800014BE0FB6F894A89580916000886180939B
:100890006000109260000FBE1092010810920008D4
:1008A000E3E0F0E089E080935700E491E695E3709F
:1008B000E150E33040F4F0E0EE0FFF1FE858FE4F48
:1008C0008081918102C080E090E1E0E0F0E8E81BE7
:1008D000F90BF695E795099511E0A0E0B1E0E8E99C
:1008E000F4E602C005900D92AE37B107D9F724E0C7
:1008F000AEE7B1E001C01D92A232B207E1F714E009
:10090000C2E2D4E004C02197FE010E943032C0321E
:10091000D107C9F70E949A1A0C944A320C9400002D
:10092000FF93EF93E0917E01F0917F01309709F002
:100930000995EF91FF910895FC018591803011F0A8
:10094000EFDFFBCF0895FF27E0E230E247FF0CC066
:10095000419597FF09C0EDE260957095809590955F
:10096000611D711D811D911D27FF02C0219530E37E
:1009700050E2AA27660F771F881F991FAA1FA41786
:1009800010F0A41B63955A95A9F7AA3008F0A95F47
:10099000A05DAF93F395611571058105910541F750
:1009A000ED3211F4EF93F395F21718F43F93F395AA
:1009B000FBCF8F91B5DFFA95E1F70895E991F991B1
:1009C0008591803021F0853219F0AADFF9CF0895A2
:1009D00020E0E89455915532C1F3503311F46894F6
:1009E00055915A3348F4505390F3220F022E220FA0
:1009F000220F200D250FF4CF0EF4219589919991A6
:100A0000533619F3533729F1533559F1BC0188276F
:100A10009927E8945C3621F48991999168945591CD
:100A2000543639F446EF7EF077FF0DC08FEF9FEF1D
:100A30000AC055374AE039F0583540E121F05236C6
:100A400042E009F00895FF93EF937DDFEF91FF916E
:100A5000B7CFFF93EF93FC0181918030B9F360DF52
:100A6000FBCFFF93EF9368DFF1CFDF93CF93CDB749
:100A7000DEB72596A3DFCF91DF910895FC012AB15F
:100A8000938D909592239AB99BB1838D892B8BB9C5
:100A90000895FC019AB1838D809589238AB99BB111
:100AA000838D892B8BB985E08A95F1F7000099B188
:100AB000838D982381E009F480E00895FC012BB137
:100AC000948D909592239BB99AB1848D892B8AB984
:100AD0000895FC012AB1948D909592239AB99BB107
:100AE000848D892B8BB90895FC019AB1848D8095F2
:100AF00089238AB99BB1848D892B8BB985E08A952E
:100B0000F1F7000099B1848D982381E009F480E029
:100B100008950F931F93CF93DF938C01EB01C801CE
:100B20000E944905882341F0209731F085E08A959D
:100B3000F1F700002197F3CFCE01DF91CF911F9104
:100B40000F9108950F931F93CF93DF938C01EB01C7
:100B5000C8010E944905811108C0209731F085E045
:100B60008A95F1F700002197F3CFCE01DF91CF9165
:100B70001F910F910895CF93DF93EC010E943E05E2
:100B8000CE01DF91CF910C9469053BB1FC01238D1F
:100B9000209523232BB93AB1238D232B2AB90C940A
:100BA0006905FC018CB3938D982B9CBB9DB3838D01
:100BB000892B8DBB0895CF93DF93EC010E94D10563
:100BC000CE01DF91CF910C94BB05FC012DB3938D29
:100BD000909592239DBBCF010C94C505FC01118219
:100BE00010821282138280E090E8958384831782BA
:100BF00010860895CF93DF93EC012E9826982F98B6
:100C000027980E94C505898D843080F44091690041
:100C1000880F22E030E0B90102C0660F771F8A9585
:100C2000E2F7CB01842B8093690010C040916A00E9
:100C30008370880F22E030E0B90102C0660F771F91
:100C40008A95E2F7CB01842B80936A009DB38B8D4C
:100C5000809589238DBBCE01DF91CF910C94EE0559
:100C6000CF93DF93EC018F8190E001968F709927ED
:100C7000288530E08217930749F4CE010E94EE05E3
:100C8000CE010E94D105CE010E94BB052FB7F8947A
:100C900098858F81891751F0FE01E90FF11D81853B
:100CA0009F5F9F709887C82FD0E002C0CFEFDFEF23
:100CB0002FBFCF3F8FEFD80781F08091070480FFCF
:100CC0000CC0DF93CF9382E892E09F938F930E94B2
:100CD00035050F900F900F900F90CE01DF91CF91BF
:100CE00008950F931F93CF938C01CAE1C15071F007
:100CF000C8010E9430068F3F2FEF920749F48FE919
:100D00009FE00197F1F700C00000F0CF8FEF9FEF59
:100D1000CF911F910F9108952F923F924F925F9222
:100D20006F927F928F929F92AF92BF92CF92DF92FB
:100D3000EF92FF920F931F93CF93DF93EC01062F57
:100D40001B828091070480FF0CC01F926F9386E97D
:100D500092E09F938F930E9435050F900F900F9014
:100D60000F908C819D818115904899F080910704A6
:100D700080FF19C18C819D819F938F938CE892E0B5
:100D80009F938F930E9435050F900F900F900F90B7
:100D90000AC19DB38B8D809589238DBB2BE0A22E3C
:100DA000BB24B39410E09924939438E0232E47E0B9
:100DB000342E56E0452E65E0562E74E0872EE3E093
:100DC0007E2EF2E06F2EA9E8CA2EA2E0DA2ECE0126
:100DD0000E94C5058FE193E00197F1F700C0000084
:100DE000CE010E945E058FE193E00197F1F700C00C
:100DF0000000CE010E943E0568E97AE3CE010E9420
:100E00008905892B11F49B826FC0E12CF12C90E5B0
:100E10009A95F1F7C8010E2C02C0959587950A9412
:100E2000E2F780FF05C0B924CE010E94690503C026
:100E3000CE010E945E0562E370E0CE010E94A20531
:100E4000892B11F46B8250C062E370E0CE010E94E6
:100E50008905892B11F47B8247C02FEFE21AF20A31
:100E600088E0E816F10499F690E59A95F1F7CE013D
:100E7000BB2019F00E94690502C00E945E0562E372
:100E800070E0CE010E94A205892B11F48B822CC048
:100E900062E370E0CE010E948905892B11F45B8228
:100EA00023C020E52A95F1F7CE010E9469059CE256
:100EB000E92EFF24F394CE010E947405882329F0C3
:100EC000E114F104C9F44B820FC0EF28E1F38CE286
:100ED000E82EFF24F394CE010E947405811114C002
:100EE000E114F104D1F53B828B81813009F049C0D6
:100EF000AA94A1103AC045C085E08A95F1F7000098
:100F000091E0E91AF108D7CFEF2869F36CE271E0BC
:100F1000CE010E94A205892B11F42B82E5CFCE01D0
:100F20000E94EE05CE010E94BB05CE010E94D105B4
:100F3000CE01DF91CF911F910F91FF90EF90DF9045
:100F4000CF90BF90AF909F908F907F906F905F9069
:100F50004F903F902F900C94710625E02A95F1F761
:100F6000000081E0E81AF108B6CF1B8280910704E7
:100F700080FF2DCFDF92CF920E9435050F900F900A
:100F800026CF8B8180618B83CE010E94C5058FE3C4
:100F90009FE10197F1F700C00000CE010E94BB0560
:100FA000CE010E94D1058FEF9FEFDF91CF911F916E
:100FB0000F91FF90EF90DF90CF90BF90AF909F90F8
:100FC0008F907F906F905F904F903F902F900895FB
:100FD0001F93CF93DF93EC01162F6DEE0E948C06CA
:100FE0008A3F910539F4612FCE01DF91CF911F9196
:100FF0000C948C06DF91CF911F9108951F920F9250
:101000000FB60F9211242F933F934F935F938F93BB
:101010009F93EF93FF9349B15091B70190910804CA
:101020002091A1013091A2012115304819F490932B
:10103000A3010FC08091A301981B933050F08091C1
:10104000A1019091A20190939E0180939D0180E265
:101050001AC12091A1013091A201369527953093B4
:10106000A2012093A10181E090E001C0880F5A9570
:10107000EAF7842349F08091A1019091A201906840
:101080009093A2018093A1018091A1019091A2016E
:1010900099278038910509F450C1A8F48032910550
:1010A00009F44BC138F4009709F447C1409709F49B
:1010B00095C0DEC08034910509F43FC180359105AB
:1010C00009F48CC0D5C0803C910531F148F48039D9
:1010D000910509F483C0803A910509F44DC0C8C058
:1010E000803D910509F47AC0803E910509F0C0C0A9
:1010F0008091A1019091A20190939E0180939D0106
:101100008091A1019091A201892F99279093A2012A
:101110008093A10183E256C080919F01811123C079
:1011200084E629B19091B801922311F48111EDC0A8
:1011300029B19091B8019223E1F08111ECC0809126
:10114000A1019091A20190939E0180939D018091B5
:10115000A1019091A201892F99279093A2018093D8
:10116000A10182E22FC080919F01823209F0E5C087
:10117000E6CF8111E2C0E3CF80919F01811125C0AC
:1011800084E629B19091B801922311F48111C9C06C
:1011900029B19091B8019223F1F08111C8C08091DA
:1011A000A1019091A20190939E0180939D01809155
:1011B000A1019091A201892F99279093A201809378
:1011C000A10181E280939F016BC080919F018132D8
:1011D00009F0B3C0E4CF8111B0C0E1CF8091A1018B
:1011E0009091A20190939E0180939D018091A10115
:1011F0009091A20180399A4A11F482E044C0209172
:10120000A1013091A2018091A1019091A201232F0F
:1012100036E026953A95E9F7217056E09695879540
:101220005A95E1F78227982F9E7F29F0982F96955F
:1012300081708927F8CF811102C081E024C080919C
:10124000A1019091A20197FF02C080E101C081E15C
:1012500080939F018091A1019091A20126E0969533
:1012600087952A95E1F79093A2018093A10118C078
:1012700010929F018091A1019091A20190939E01F3
:1012800080939D0180E88093A0019BB18091B8017B
:10129000282F209592239BB99AB1892B8AB92EC009
:1012A0002091A1013091A2018091A401E82FF0E0EA
:1012B000E356FE4F21878F5F8F708093A40190E0EB
:1012C00001968F7099273091A501432F50E0841724
:1012D000950769F42DB38091B801482F40952423D8
:1012E0002DBB9BB194239BB99AB1892B8AB980916C
:1012F000A401831303C080E48093A00180E090E800
:101300009093A2018093A10118C095E09A95F1F7FE
:101310000000815006CF25E02A95F1F700008150AA
:1013200007CF95E09A95F1F7000081502ACF25E08C
:101330002A95F1F7000081502BCFFF91EF919F91FB
:101340008F915F914F913F912F910F900FBE0F9012
:101350001F9018951F920F920FB60F9211242F9382
:101360003F934F935F938F939F93EF93FF9349B175
:1013700050919A0190910804209184013091850147
:101380002115304819F4909386010FC08091860191
:10139000981B933050F08091840190918501909337
:1013A00081018093800180E21AC1209184013091F3
:1013B000850136952795309385012093840181E03E
:1013C00090E001C0880F5A95EAF7842349F0809194
:1013D00084019091850190689093850180938401A8
:1013E000809184019091850199278038910509F4B5
:1013F00050C1A8F48032910509F44BC138F400972C
:1014000009F447C1409709F495C0DEC080349105C6
:1014100009F43FC18035910509F48CC0D5C0803CEA
:10142000910531F148F48039910509F483C0803A7F
:10143000910509F44DC0C8C0803D910509F47AC0FA
:10144000803E910509F0C0C0809184019091850192
:101450009093810180938001809184019091850116
:10146000892F9927909385018093840183E256C048
:1014700080918201811123C084E629B190919B0162
:10148000922311F48111EDC029B190919B01922317
:10149000E1F08111ECC080918401909185019093DD
:1014A0008101809380018091840190918501892F31
:1014B0009927909385018093840182E22FC08091C7
:1014C0008201823209F0E5C0E6CF8111E2C0E3CFAC
:1014D00080918201811125C084E629B190919B0100
:1014E000922311F48111C9C029B190919B019223DB
:1014F000F1F08111C8C08091840190918501909391
:101500008101809380018091840190918501892FD0
:101510009927909385018093840181E280938201D1
:101520006BC080918201813209F0B3C0E4CF811198
:10153000B0C0E1CF809184019091850190938101A9
:1015400080938001809184019091850180399A4A2D
:1015500011F482E044C02091840130918501809192
:10156000840190918501232F36E026953A95E9F77D
:10157000217056E0969587955A95E1F78227982F26
:101580009E7F29F0982F969581708927F8CF811139
:1015900002C081E024C0809184019091850197FF71
:1015A00002C080E101C081E18093820180918401C9
:1015B0009091850126E0969587952A95E1F790937D
:1015C00085018093840118C010928201809184016A
:1015D00090918501909381018093800180E88093B0
:1015E00083019BB180919B01282F209592239BB969
:1015F0009AB1892B8AB92EC020918401309185013E
:1016000080918701E82FF0E0E058FE4F21878F5F3F
:101610008F708093870190E001968F7099273091A9
:101620008801432F50E08417950769F42DB380910A
:101630009B01482F409524232DBB9BB194239BB93C
:101640009AB1892B8AB980918701831303C080E402
:101650008093830180E090E89093850180938401DA
:1016600018C095E09A95F1F70000815006CF25E06B
:101670002A95F1F70000815007CF95E09A95F1F790
:10168000000081502ACF25E02A95F1F70000815013
:101690002BCFFF91EF919F918F915F914F913F9150
:1016A0002F910F900FBE0F901F901895EDE9F1E06C
:1016B000118210821282138220E030E83583248365
:1016C000168291E0918F128E82E0838F948FE0E8F2
:1016D000F1E01182108212821382358324831682F4
:1016E00093E0918F828F88E0838F84E0848F0895C8
:1016F000E62FF0E034E0F595E7953A95E1F7E770ED
:101700006F70823079F08330C1F0813011F5F0E0F4
:1017100024E0EE0FFF1F2A95E1F7E60FF11DE05ED2
:10172000FA4F15C0F0E094E0EE0FFF1F9A95E1F735
:10173000E60FF11DE056FB4F0AC0F0E084E0EE0F2B
:10174000FF1F8A95E1F7E60FF11DE05EFB4F8491E4
:10175000089580E808950F931F93CF93DF938C0132
:10176000EB0169EEFC01808191810E948C06F801F9
:10177000808191810E9471068883F8018081918126
:101780000E9471068983F801808191810E9471060F
:101790008A8399279F938F9389811F928F93888142
:1017A0001F928F938DE094E09F938F930E94350555
:1017B0008DB79EB708960FB6F8949EBF0FBE8DBF2B
:1017C000DF91CF911F910F910895E7EDF1E0119214
:1017D000119281E0E73EF807D1F70895CF93DF93A8
:1017E000EC011B821A821C821D820E94E50B8881FB
:1017F0009981DF91CF910C94FA051F93CF93DF93DA
:10180000FC0184810E94780B87FD20C0182F1F7077
:10181000C82FD0E094E0D595C7959A95E1F7612F50
:101820008C2F0E947621811111C0CC0FDD1FC9526F
:10183000DE4F81E090E002C0880F991F1A95E2F711
:1018400028813981822B932B99838883DF91CF91D3
:101850001F9108951F93CF93DF93FC0184810E9411
:10186000780B87FD22C0182F1F70C82FD0E094E09E
:10187000D595C7959A95E1F7612F8C2F0E94762117
:10188000882399F0CC0FDD1FC952DE4F81E090E034
:1018900002C0880F991F1A95E2F7809590952881CC
:1018A00039818223932399838883DF91CF911F917C
:1018B000089589EC91E00E94EE0B8BEB91E00C9483
:1018C000EE0B809107048160809307040C94E50B74
:1018D000E82FF0E0EE0FFF1FE952FE4F808191816B
:1018E00008950C94E50BE82FF0E083E0EE0FFF1F66
:1018F0008A95E1F77770E70FF11D94E0EE0FFF1F77
:101900009A95E1F76F70E60FF11DEE0FFF1FE050A3
:10191000F8498591949108958091BA010895FC0148
:101920008481823070F0843061F062FB992790F9F5
:1019300060FD926061FD9460692F808191810C94BB
:10194000E8070895CF93C82F682F89EC91E00E9493
:101950008F0C6C2F8BEB91E0CF910C948F0CCF926E
:10196000DF92EF92FF920F931F93CF93DF936C015F
:101970008B010E94AD2D7C01F601808191810E9436
:101980003006EC01019631F4C7010E94C52D801785
:10199000910790F3CE01DF91CF911F910F91FF90AE
:1019A000EF90DF90CF9008950F931F93CF93DF9325
:1019B000FC0180819181DC0112962C912131F9F09A
:1019C0008F0162EF0E948C068F3FBFEF9B07D1F023
:1019D0008A3F9105D1F464EF71E0C8010E94AF0C19
:1019E0008F3F2FEF9207A1F0D82FCC2764EF71E043
:1019F000C8010E94AF0CDE01A82BCD010BC08DEFFA
:101A00009FEF08C08FEF9FEF05C08EEF9FEF02C0E2
:101A100080E090E0DF91CF911F910F910895CF93D7
:101A2000862F90E0FC017C97E834F105A0F5E65C98
:101A3000FF4F0C94303285E53EC08AE53CC08BE513
:101A40003AC08CE538C08DE536C08EE534C08FE5F0
:101A500032C080E630C081E62EC082E62CC083E62C
:101A60002AC08FE628C081E726C082E724C084E729
:101A700022C085E720C087E71EC088E71CC08AE730
:101A80001AC08CE718C08FE716C080E714C089E73A
:101A900012C08BE710C0C62F1F926F9383EF92E0A6
:101AA0009F938F930E9435050F900F900F900F908A
:101AB0008C2F01C084E5CF910895CF93DF93EC0183
:101AC00099859230A9F128F4992341F09130C9F019
:101AD00045C09330B1F19430D9F140C0603E21F05F
:101AE000613E21F482E02BC081E029C067FD04C083
:101AF000CE010E94FD0B33C06F77CE010E942A0CED
:101B00002EC0663359F118F46A3229F427C06A3AB4
:101B100029F1663B19F167FD05C0CE010E940F0D4A
:101B2000682F12C06F77CE010E940F0D682F13C06F
:101B30006D3121F06D3991F484E001C083E0898733
:101B40000EC0653459F465E5CE010E94FD0B06C058
:101B5000653C21F465E5CE010E942A0C198680E0DF
:101B6000DF91CF910895862F90E0FC013397E13803
:101B7000F10508F048C0EE57FF4F0C94303289E170
:101B8000089587E108958FE1089587E2089580E63A
:101B9000089582E608958CE5089583E508958FE21F
:101BA000089589E3089587E308958FE3089587E40E
:101BB00008958FE4089586E508958EE508958FE7EA
:101BC000089580E0089585E608958EE608958FE6ED
:101BD000089580E3089588E3089580E4089588E4F3
:101BE000089580E5089587E508958FE5089588E1D3
:101BF000089588E0089580E2089580E108958DE6D3
:101C0000089588E20895862F8F7708958FE00895CC
:101C1000623309F44AC010F5643209F44CC080F410
:101C20006C3109F44CC028F46B3109F04AC08FE1E3
:101C300008956D31F1F1633209F043C087E20895F0
:101C40006B3209F440C020F46A32D9F588E4089573
:101C50006C3229F16D32A9F581E508956234E9F01D
:101C600048F46433B1F0B8F06A3309F16C3349F5E4
:101C700080E308956B34B9F030F4633491F0643448
:101C800001F585E608956D34C1F06136D1F48AE638
:101C9000089580E1089588E1089580E2089588E23A
:101CA000089588E3089580E4089580E5089587E520
:101CB00008958FE5089587E108958EE608958FE6EB
:101CC0000895862F089588E008956B35C9F068F46B
:101CD0006131F1F020F46E30C9F484E50895633188
:101CE00069F0643599F48BE508956D3559F050F03D
:101CF000623651F06C3751F487E7089581E1089519
:101D00008DE508958AE608958EE00895862F08955A
:101D10008FE00895613131F0613411F48CE708955A
:101D2000862F089583E108951F93CF93DF93EC01ED
:101D3000162FEA858E2F90E08B30910508F0D2C0E7
:101D4000FC01ED5FFE4F0C9430328A819B818059FB
:101D50009B4A029720F4CE010E94650E182F14387A
:101D6000A9F030F4103881F0133891F462E090C09B
:101D7000113E41F0103F21F0103E51F482E08FC03F
:101D800081E08DC084E08BC089E089C06FE780C0AE
:101D90001A8617FD02C0612F98C00E94E50B87EEDE
:101DA00092E063C08A819B8180599B4A029720F40C
:101DB000CE010E948A0E182F193509F493C0103FE6
:101DC00019F0123119F48EC083E069C01A8617FD2C
:101DD00005C0612FCE010E94B30D76C00E94E50BB5
:101DE0008DED92E042C08A819B8180599B4A029787
:101DF00020F4CE010E94650E182F133821F01438FC
:101E000021F46FE755C062E053C01A8617FD02C087
:101E1000612F64C00E94E50B1F921F938EEC92E02D
:101E20009F938F930E9435050F900F900F900F9006
:101E300022C08A819B8180599B4A029720F4CE015F
:101E40000E948A0E182F1A86123109F44CC01935D7
:101E500009F449C017FD05C0612FCE010E94B30DE2
:101E60003CC00E94E50B81EC92E09F938F930E940F
:101E700035050F900F908FEF37C0643121F0603F30
:101E800089F586E00CC085E00AC0673759F560E047
:101E9000CE010E94FD0B26C0643121F587E08A87C0
:101EA00022C0603FF9F488E0FACF6737D9F460E0E8
:101EB000CE010E942A0C16C0603F11F48AE0EFCFD9
:101EC0001A86CE010E94080E682FCE010E94FD0BDB
:101ED0000AC01A86CE010E94080E682FCE010E9409
:101EE0002A0C01C01A8680E0DF91CF911F910895DE
:101EF0006C3551F018F4633169F00AC0663731F07F
:101F00006E3731F486E7089581E508958EE70895E8
:101F1000862F08958DE50895663809F466C058F552
:101F2000673609F450C0A0F46C3509F464C040F47D
:101F3000683009F464C0673509F05FC08CE5089526
:101F4000643609F444C0653609F057C08DE608953B
:101F5000673709F44EC038F46D36B9F16E3609F0C2
:101F60004CC085E608956438A1F1E8F56C3709F0B6
:101F700044C088E608956C38A1F178F4693869F1B5
:101F800030F4673841F16838C1F58EE708956A3852
:101F900031F16B3891F584E008956F3881F030F4B9
:101FA0006D3859F06E3849F587E608956139F9F0D2
:101FB00040F0623911F589E0089587E708958FE7C9
:101FC00008958BE7089582E6089584E608958EE6E5
:101FD00008958CE7089582E008958CE0089583E0E9
:101FE000089585E0089588E0089580E1089581E0EE
:101FF000089588E5089583E50895862F089586E776
:102000000895CF93DF93EC016F3B41F028F486E510
:10201000860F823070F402C06C3F59F41B8684EB4B
:1020200092E09F938F930E9435050F900F908FEF52
:10203000C1C08B85813009F44DC038F0823009F47D
:1020400086C0833009F4A1C0B4C08A819B818239E3
:102050002BEA920721F4CE010E94780F06C0813945
:102060009B4A21F4CE010E948C0F682F663809F13B
:1020700068F46338D1F020F4603819F582E07FC04D
:102080006438A9F06538E9F468E61DC06C38A9F039
:1020900030F4673881F06B38A1F461E014C06D381A
:1020A00071F0603F71F481E06AC062E00CC06FE7DC
:1020B0000AC068E708C060E006C069E004C06AE0E2
:1020C00002C067FD04C0CE010E94FD0B72C087EA0A
:1020D00092E036C01B868A819B8182392BEA920767
:1020E00021F4CE010E94780F06C081399B4A21F469
:1020F000CE010E948C0F682F862F90E0FC01E358E0
:10210000F109EB30F105A0F4E25FFE4F0C943032A0
:1021100062E010C06FE70EC068E60CC068E70AC056
:1021200060E008C061E006C069E004C06AE002C087
:1021300067FD04C0CE010E942A0C3BC08DE992E0ED
:102140009F938F930E9435050F900F9032C0653298
:1021500079F030F4663171F06E3199F460E00BC0C3
:10216000663221F0603F69F483E009C06DE503C089
:1021700063E501C061E5CE010E94FD0B04C08B87C1
:1021800018C00E94E50B1B8614C06E3169F020F464
:102190006631B9F761E509C0653221F0663289F729
:1021A0006DE503C063E501C060E0CE010E942A0C2A
:1021B000EACF80E0DF91CF9108958F929F92AF9206
:1021C000BF92CF92DF92EF92FF920F931F93CF9324
:1021D000DF9300D000D01F92CDB7DEB78C01DC01B9
:1021E000ED91FC918381882391F1E080F180D3808F
:1021F0000E94AD2DFF92EF921F92DF929F938F93DB
:1022000086EF93E09F938F930E943505D801ED915F
:10221000FC911197838180750FB6F894DEBF0FBED5
:10222000CDBF79F418968C9118978B3019F48CE007
:1022300018968C938381823021F48DE0D801189612
:102240008C931382D801ED91FC9111821082D801F8
:10225000ED91FC9111978281882381F192811596ED
:102260008C91981759F1E080F180D2800E94AD2DB9
:10227000FF92EF921F92DF929F938F938FED93E0E7
:102280009F938F930E943505F80185810FB6F894CE
:10229000DEBF0FBECDBF0190F081E02D85FF03C0F2
:1022A000928194FDA1C584FD9CC5D801ED91FC915E
:1022B0001197828115968C9311821082D8011896FD
:1022C000EC918E2F90E08E30910508F0E9C5FC016D
:1022D000E75EFE4F0C9430320E94AD2D9F938F939A
:1022E00083ED93E09F938F930E9435050E94AD2D5F
:1022F000F80197838683808191810E94DB0581E0CC
:10230000D80118968C936BC0F801808191810E944E
:1023100030060196C9F7D80116968D919C911797B2
:102320000E94C52D893B9B4008F4BAC582E041C597
:102330000E94AD2D9F938F938EEC93E09F938F938C
:102340000E9435056FEFD8018D919C910E948C06FB
:102350000F900F900F900F908A3F910511F486E037
:1023600028C583E06FC3F801808191810E94E50553
:102370002E98269A2F98279A0E94AD2DD80117964D
:102380009C938E93169784E05EC3F80186819781B3
:102390000E94C52D853F914008F482C585E052C357
:1023A0002E9826982F982798F801808191810E9475
:1023B000EE05D8018D919C910E94DB050E94AD2D08
:1023C0009F938F9389EC93E09F938F930E943505A1
:1023D0000E94AD2DF8019783868386E080870F9059
:1023E0000F900F900F905CC5D8018D919C910E9429
:1023F0003006019609F454C50E94AD2D9F938F932A
:1024000084EC93E09F938F930E9435050E94AD2D3D
:10241000F8019783868387E0E1CFD80116968D91E6
:102420009C9117970E94C52D853F914018F089E037
:10243000F8018087D8018D919C910E943006019609
:1024400009F42EC50E94AD2D9F938F938FEB93E0DF
:102450009F938F930E9435050E94AD2DF8019783BD
:10246000868388E0BBCFD80116968D919C911797F3
:102470000E94C52D853F914018F089E0F8018087C2
:10248000D8018D919C910E943006019609F408C5EF
:102490000E94AD2D9F938F938AEB93E09F938F9330
:1024A0000E94350589E0F80199CFC8010E94D40C3B
:1024B000D80113969C938E9312970E94AD2D9F93F3
:1024C0008F9385EB93E09F938F930E943505F801DE
:1024D000828193810F900F900F900F90009711F4CD
:1024E00082E010C08F3FBFEF9B0711F481E044C032
:1024F0009C012D5F3F4F2230310590F38F3F9105B6
:1025000029F484E0D80114968C9372C09C0125585C
:102510003B4A2230310508F49FC48239BBEA9B074D
:1025200009F49AC49C0120593B4A22303105F8F441
:1025300088EA93E09F938F930E94350582E0F8012B
:10254000848360EF808191810E948C060F900F90B0
:102550008A3F9105F1F562E8D8018D919C910E9426
:102560008C068A3F9105A9F584EA93E06EC4803B0E
:10257000BFEB9B0721F483E0F801848339C08827EF
:102580008115FBEA9F0709F4ABCF81152FEB92076A
:1025900091F381159F4779F38CE793E09F938F9395
:1025A0000E94350560EFD8018D919C910E948C06A8
:1025B0000F900F908A3F910509F04EC462E0F80138
:1025C000808191810E948C068A3F910509F044C464
:1025D00087CF80EA93E09F938F930E9435050F90F9
:1025E0000F90F8018281938181399B4A09F40EC4CE
:1025F000F801228133812E3FFFEF3F0751F02D3F3D
:102600004FEF340749F02115310549F040E251E020
:1026100008C041E251E005C04BE151E002C047E291
:1026200051E0D80114968C91813049F0823051F0FC
:10263000833059F0843061F08CE391E00BC080E38B
:1026400091E008C08DE291E005C083E391E002C013
:1026500081E491E05F934F939F938F933F932F93E8
:102660008CE693E09F938F930E9435058AE0F801F2
:10267000808781C30E94AD2D9F938F9387E693E05F
:102680009F938F930E9435050F900F900F900F909E
:10269000D80114968C91833031F0843079F08230F7
:1026A00009F07CC106C068EFF801808191810E9429
:1026B0008C060E94E21F0E94A20C70C165EFD80137
:1026C0008D919C910E948C066AEEF8018081918127
:1026D0000E948C06BE016F5F7F4FC8010E94AB0B4A
:1026E00080E693E09F938F930E94350568EED801B2
:1026F0008D919C910E948C0660E0F801808191810F
:102700000E948C0666EED8018D919C910E948C06E9
:1027100066EEF801808191810E948C0666EED801F8
:102720008D919C910E948C06BE016F5F7F4FC80106
:102730000E94AB0B0F900F908981882309F47AC017
:102740008A81882309F476C089E593E09F938F936B
:102750000E94350566EEF801808191810E948C0609
:1027600068EED8018D919C910E948C0660E0F80182
:10277000808191810E948C0668EED8018D919C9198
:102780000E948C0663E0F801808191810E948C0692
:1027900068EED8018D919C910E948C0662E0F80150
:1027A000808191810E948C0668EED8018D919C9168
:1027B0000E948C0661E0F801808191810E948C0664
:1027C00066EED8018D919C910E948C0668EEF8010E
:1027D000808191810E948C0663E0D8018D919C914B
:1027E0000E948C0668EEF801808191810E948C061F
:1027F00061E0D8018D919C910E948C0668EEF801F1
:10280000808191810E948C0662E0D8018D919C911B
:102810000E948C0668EEF801808191810E948C06EE
:1028200063E0D8018D919C910E948C0689E0F801AB
:10283000848781C082E593E09F938F930E94350542
:1028400063EFD8018D919C910E948C0668ECF80191
:10285000808191810E948C0663EFD8018D919C91BB
:102860000E948C0664E6F801808191810E948C06AA
:1028700063EFD8018D919C910E948C0660E5F80170
:10288000808191810E948C06C8010E94D40C292F5E
:1028900030E00F900F902330310511F080E001C03F
:1028A00083E0D8011C968C938BE493E09F938F93E5
:1028B0000E94350563EFF801808191810E948C06AA
:1028C00068ECD8018D919C910E948C0663EFF80111
:1028D000808191810E948C0668ECD8018D919C9139
:1028E0000E948C0663EFF801808191810E948C0622
:1028F00060E5D8018D919C910E948C06C8010E94D0
:10290000D40C292F30E00F900F902430310511F0B6
:1029100080E001C084E0F801848781110EC084E466
:1029200093E09F938F930E94350566EFD8018D91B8
:102930009C910E948C060F900F9064EFF8018081AB
:1029400091810E948C06BE016F5F7F4FC8010E947B
:10295000AB0BD8011C968C91893049F0833051F033
:10296000843059F0882361F083E291E00BC08FE45A
:1029700091E008C087E491E005C088E591E002C0DD
:1029800081E691E09F938F9388E393E09F938F93E9
:102990000E9435050F900F900F900F908BE0F8017B
:1029A00080870E94AD2D9F938F9383E393E09F9345
:1029B0008F930E9435050F900F900F900F90D801C4
:1029C0008D919C910E9430064C01019609F468C2D9
:1029D000F8018481843069F18114910421F0FFEFC2
:1029E0008F16910469F40E94E50B0E940C238BE280
:1029F00093E09F938F930E9435050F900F9050C2E4
:102A0000823069F0833081F0813009F049C2682D4D
:102A1000C8010E945D0D8F3F09F042C212C0682DAF
:102A2000C8010E94940EF7CF682DC8010E940110C2
:102A3000F2CFF801808191810E9471066C010196AC
:102A400029F48CE0D80118968C932AC2F801808171
:102A500091810E9471067C01019699F3D8011C9620
:102A60008C91FE0131965F01853028F4833030F47B
:102A7000882321F0DEC08930A1F0DBC0D8011D968B
:102A80009C911D97987F282D2770922B1D969C93C3
:102A900084FE02C0DD24DA9485FEC6C0FF24FA94C9
:102AA000C3C0F8013585C40188749927883491051D
:102AB00009F0ABC0C1FEA9C0F0E38F229924959420
:102AC00087949594879420E3C222DD2454E0D59422
:102AD000C7945A95E1F7C828D92842E0C416D10412
:102AE000E1F183E0C816D10409F478C0CA94CD2876
:102AF00009F0C7C1E6FC17C0A701487055278E2D05
:102B00008F70E7FE07C0452B11F420E001C020EFD5
:102B1000822B0AC0452B11F420E001C020EF982F32
:102B2000922B80E002C080E090E0E4FE05C03860B7
:102B3000D8011D963C9303C0377FF8013587D80133
:102B40001D962C911D97E5FE04C020611D962C93C7
:102B50009AC12F7EF801258796C1E0FE05C030643A
:102B6000D8011D963C9303C03F7BF8013587D801FF
:102B70001D968C911D97E1FE04C080681D968C9374
:102B800003C08F77F8018587D8011D968C911D971A
:102B9000E2FE04C080621D968C9303C08F7DF80115
:102BA0008587D8011D968C911D97E3FE04C0806433
:102BB0001D968C9303C08F7BF8018587D8011D96E5
:102BC0008C911D97E4FE04C080681D968C9303C011
:102BD0008F77F801858780E090E055C1C70124E038
:102BE000959587952A95E1F7E7FE03C0806F90E001
:102BF00003C0982F9F7080E0387F2E2D2770E32E22
:102C0000E22AD8011D96EC923EC1387F882D87704C
:102C1000382BF801358784FE02C0DD24DA9485FE66
:102C20004DC0FF24FA944AC0833049F08430C9F083
:102C300045C0833079F4E12CF12CC12CD12CD80182
:102C40008D919C910E9471068F3FBFEF9B07B1F160
:102C5000982F35C0843009F014C1E12CF12CC12C1F
:102C6000D12CF801808191810E947106AC018F3FC7
:102C7000FFEF9F0719F183FD02C080E001C080EFE4
:102C8000942F9F70982BD8011D962C911D9744FF6F
:102C900004C028601D962C9303C0277FF801258768
:102CA000D8011D962C911D9745FF04C020611D96EB
:102CB0002C9305C02F7EF801258701C090E085E0A8
:102CC000D5011D928A95E9F7F8018585898380E011
:102CD000F0E8CF16D1044CF4960141E8C4164FEF4A
:102CE000D40624F421E83FEF01C02FE72A83A0E8AF
:102CF000EA16F10454F49701B1E8EB16BFEFFB06B6
:102D000014F421E83FEF219501C021E82B8390388E
:102D100011F0919501C09FE79C83803809F481E808
:102D20008D83C5010E94372089818093BA011F924B
:102D30008F938D81282F082E000C330B3F938F9398
:102D40008C81282F082E000C330B3F938F938B819F
:102D5000282F082E000C330B3F938F938A81282F46
:102D6000082E000C330B3F938F938CE093E09F93DE
:102D70008F930E9435050FB6F894DEBF0FBECDBF0E
:102D80008FC00E94AD2D9F938F9387E093E09F9318
:102D90008F930E9435056EEFD8018D919C910E9412
:102DA0008C060F900F900F900F908A3A910521F4A6
:102DB00089E0F801808774C00E94AD2D9F938F93A6
:102DC00082E093E09F938F930E943505C8010E9493
:102DD000EE0B0E94E50B0E940C23D80118961C9262
:102DE000FECA828185FF61CAD80118968C918B300A
:102DF00009F05BCA88ED93E09F938F930E9435059D
:102E00008CE0F80180870F900F904FCA60EFF801B7
:102E1000808191810E948C068A3F9105A1F463E034
:102E2000D8018D919C910E948C068A3F910559F49E
:102E30008CE993E09F938F930E94350583E0D8013E
:102E400014968C9306C088E993E09F938F930E9419
:102E500035050F900F90CCCB60EFF8018081918108
:102E60000E948C068A3F910509F03ACB63E0D801B5
:102E70008D919C910E948C068A3F910509F030CB80
:102E80007ACB90E080E025E0D5011D922A95E9F704
:102E9000F80125852983E12CF12CC12CD12C1CCFE4
:102EA00081E00F900F900F900F900F90DF91CF91D6
:102EB0001F910F91FF90EF90DF90CF90BF90AF9058
:102EC0009F908F90089589EC91E00E94DD108BEB2C
:102ED00091E00C94DD10E9ECF1E08DE991E0918353
:102EE00080831382128214821582108611861286C4
:102EF0001386148615860E94E50BEBEBF1E080E863
:102F000091E091838083138212821482158210864D
:102F1000118612861386148615860C94E50B809113
:102F20000B030895CF93DF9300D01F92CDB7DEB788
:102F300020911904243021F523E029839B838A837F
:102F400082E08093E9008FEF9091E800815095FD39
:102F500006C095ED9A95F1F700008111F5CF8091AB
:102F6000E80085FF0DC040E050E063E070E0CE0176
:102F700001960E944E1C8091E8008E778093E800B5
:102F80000F900F900F90DF91CF910895CF93DF9323
:102F900000D01F92CDB7DEB720911904243061F51F
:102FA00019821A821B8222E029838138910520F040
:102FB000805891099B838A8382E08093E9008FEF98
:102FC0009091E800815095FD06C095ED9A95F1F736
:102FD00000008111F5CF8091E80085FF0DC040E031
:102FE00050E063E070E0CE0101960E944E1C80919B
:102FF000E8008E778093E8000F900F900F90DF919C
:10300000CF91089520911904243051F522E02093A6
:10301000E9002FEF3091E800215035FD06C035ED75
:103020003A95F1F700002111F5CF2091E80025FF36
:1030300017C020911001222341F021E02093F100DC
:1030400040E050E065E070E004C040E050E063E044
:1030500070E00E944E1C8091E8008E778093E8001B
:103060000895CF93DF9320911904243009F04AC0CA
:10307000EC01809111018823E1F0809112018823F5
:10308000C1F081E08093E90081E8815049F090919E
:10309000E80095FD05C09AE29A95F1F700C0F5CFDA
:1030A0008091E80085FF2EC040E050E060E270E0D3
:1030B00019C081E08093E90081E8815059F0909136
:1030C000E80095FD07C0EFE3F1E03197F1F700C0AC
:1030D0000000F3CF8091E80085FF14C040E050E08D
:1030E00068E070E0CE010E944E1C8091E8008E776F
:1030F0008093E80080E2FE01ABEEB2E001900D9219
:103100008A95E1F7DF91CF910895CF93C091E901BE
:10311000C1110BC00E94B92D643C79408105910515
:1031200020F081E08093E901C1E08C2FCF910895D8
:10313000FF920F931F93CF93DF93D82F0FB607FE05
:1031400083C080911904843081F08091030190E064
:1031500001962091050130E0822393232091040100
:1031600030E08217930709F0C9C00E9485188111C9
:1031700010C08091030190E001962091050130E09C
:10318000822393232091040130E08217930709F0F2
:10319000B5C00E94AD2D8C01C091E900CF70909117
:1031A000EC00892F817090FD80E8C82B83E080932C
:1031B000E90085E0F82E8091EB0085FD42C080910A
:1031C000EB0080FF3EC08091EE0087FF3AC0809107
:1031D000040190910301981709F457C09091E800F9
:1031E00095FF8AC0E0910101F0910201E80FF11D05
:1031F00020818F5F909105018923809304012093A2
:10320000F1008091E80085FDE2CF8091E80080FF29
:10321000DECF8091E8008E778093E800F092000185
:10322000D6CF8091030190E001962091050130E016
:10323000822393232091040130E08217930709F43D
:1032400048C0CF70C093E90040910301842F90E003
:1032500001962091050130E08223932320910401FF
:1032600030E08217930709F44CC0E0910101F0911E
:103270000201E40FF11DD083809103018F5F9091D3
:1032800005018923809303013CC08091E80085FFFC
:1032900033C0D093F10081E09091F200992391F036
:1032A0009091E80090FF0EC09091E80095FF03C058
:1032B0001092F100F9CF9091E8009E779093E8008A
:1032C000F0920001882309F4ACCFCF70C093E900DD
:1032D00018C080910001882309F4B3CF0E94AD2D5E
:1032E0009C018017910711F4890165CF909100012D
:1032F000915090930001F8CF80E0CECF4091030130
:10330000B4CF80E0DF91CF911F910F91FF9008958E
:10331000089542E261EC81E00E94C71B42E061EC4B
:1033200082E00E94C71B42E261EC83E00C94C71B61
:1033300080911B04833009F453C030F4813071F064
:10334000823009F4BAC008958A3009F4A6C08B30DF
:1033500009F478C0893009F0C8C020C080911A04EF
:10336000813A09F0C2C08091E800877F8093E8002D
:1033700080911E0490911F04892B21F460E28BEE52
:1033800092E003C060E080E090E070E00E949B1C4F
:103390008091E8008B778093E800089580911A046B
:1033A000813209F0A2C080911E0490911F04892BE4
:1033B00009F09BC08091E800877F8093E8008091AE
:1033C000E80082FD05C0809119048111F8CF8DC0FD
:1033D0008091F10080930B038091E8008B7781C08E
:1033E00080911A04813A09F080C080911E04909166
:1033F0001F04892BA1F48091E800877F8093E80067
:103400008091E80080FFFCCF809111018093F10052
:103410008091E8008E778093E8000E94FC1B8091E9
:103420001E0490911F04019709F05FC08091E8008D
:10343000877F8093E8008091E80080FFFCCF809137
:1034400010014AC080911A04813209F04EC0809167
:103450001E0490911F04892B69F48091E800877FF6
:103460008093E8000E94FC1B80911C048093110152
:103470000E940C2380911E0490911F040197A9F5CE
:103480008091E800877F8093E8000E94FC1B809178
:103490001C04809310010C940C2380911A04813237
:1034A00021F58091E800877F8093E8000E94FC1B53
:1034B00080911D0480930C03089580911A04813A31
:1034C000A1F48091E800877F8093E8008091E80074
:1034D00080FFFCCF80910C038093F1008091E80085
:1034E0008E778093E8000C94FC1B089580910B0369
:1034F0008093EA0110920B030E94710C0C940C2330
:103500000C94761A0E94592D80911704882329F073
:103510000E94662D81110C94B11B08950E947B2D91
:103520008091EA0180930B0308950C948E1A0895FC
:103530000C94971ACF9384B7877F84BF0FB6F89403
:10354000A89580916000886180936000109260006F
:103550000FBE90E080E80FB6F894809361009093DE
:1035600061000FBE88E998E10E94182D86E091E085
:103570000E94DD1F80EC95E00E949C040E94590C83
:103580000E94B4200E94B41E0E94071F78940E94DB
:10359000B62080911904843029F00E94C21F0E9435
:1035A000971AF7CF8EEA95E00E949C040E94981A21
:1035B00080EA95E00E949C04C3E080911904853064
:1035C00019F40E94821AF9CF0E94422D0E94BA205B
:1035D0002091E4003091E5008091E7019091E801AD
:1035E0002817390709F464C08091E4009091E50040
:1035F0009093E8018093E7010E948518882309F4DD
:1036000057C080911904843009F052C08091E900BC
:103610008F702091EC00922F917020FD90E8892B03
:10362000C093E9009091EB0090FF3FC09091EE00B5
:1036300097FF3BC09091040120910301291709F1E4
:103640002091E80025FF1DC0E0910101F0910201E9
:10365000E90FF11D30819F5F209105019223909326
:1036600004013093F1009091E80095FDE3CF909133
:10367000E80090FFDFCF9091E8009E779093E800FC
:10368000D9CF9091F200992381F09091E80090FFBA
:103690000CC09091E80095FF03C01092F100F9CFA3
:1036A0009091E8009E779093E8008F708093E900F6
:1036B0000E94C21F82CF292F332723303105C9F042
:1036C00060F42130310581F02230310509F041C02C
:1036D00084E590E02DE136E040C021323105E1F093
:1036E0002232310531F135C082E190E021E736E048
:1036F00034C099278130910549F028F0029749F5A7
:10370000E9EDF5E005C0E9E1F6E002C0EFE0F6E042
:10371000849190E09F0121C063307105D0F4660F61
:10372000771FFB01EE58FE4F2081318189E090E048
:1037300014C06330710568F4FB01EE0FFF1FE459FC
:10374000FE4F20813181FB01E759FE4F808190E0DF
:1037500004C080E090E020E030E0FA013183208373
:10376000089584E089BD86E089BD09B400FEFDCFDF
:103770008091D8008F7D8093D8008091E000826096
:103780008093E0008091E00081FDFCCF0895982FA8
:10379000953068F59093E900981739F07091EC0036
:1037A0002091ED005091F00003C0242F762F50E0BF
:1037B00021FD02C09F5FECCF3091EB003E7F309344
:1037C000EB003091ED003D7F3093ED003091EB0048
:1037D00031603093EB007093EC002093ED00509338
:1037E000F0002091EE0027FDE5CF80E008958F7076
:1037F0008093E90081E0089580911A0487FF11C049
:103800008091E80082FD05C0809119048111F8CFF4
:1038100011C08091E8008B770BC080911904882338
:1038200049F08091E80080FFF8CF8091E8008E7722
:103830008093E80008952091E4003091E50095E63A
:103840004091EC00842F817040FF23C08091E800FC
:1038500080FD1DC080911904882399F0853099F06E
:103860008091EB0085FD11C04091E4005091E5008E
:103870002417350729F3915011F09A01E1CF84E024
:10388000089582E0089583E0089581E0089580E03E
:1038900008954091E80042FFDDCF0895CF92DF9276
:1038A000EF92FF920F931F93CF93DF93EC018B0165
:1038B0007A010E941B1C811135C0E114F10439F01A
:1038C000F70180819181081B190BC80FD91FC12CEA
:1038D000D12C0115110529F18091E80085FD18C052
:1038E0008091E8008E778093E8000E94C21FE11467
:1038F000F10449F0F70180819181C80ED91ED1826F
:10390000C08285E00FC00E941B1C882311F30AC0EF
:1039100089918093F10001501109FFEFCF1ADF0A5E
:10392000D8CF80E0DF91CF911F910F91FF90EF9062
:10393000DF90CF9008952091200430912104261724
:10394000370748F06115710539F42091E8002E77AA
:103950002093E80001C0B901FC0120E06115710568
:1039600061F1809119048823D9F18530D9F18091D2
:10397000E80083FD39C08091E80082FD2BC0809172
:10398000E80080FFEBCF8091F20090E061157105B7
:1039900051F08830910538F421912093F100615065
:1039A00071090196F3CF21E0089709F020E080919A
:1039B000E8008E778093E800D1CF2111D2CF0AC0E2
:1039C00080911904882361F0853061F08091E800CE
:1039D00083FD0AC08091E80082FFF2CF80E0089565
:1039E00082E0089583E0089581E008952091200405
:1039F000309121042617370748F06115710539F415
:103A00002091E8002E772093E80001C0B901FC0165
:103A100020E06115710579F180911904882309F47A
:103A20003DC0853009F43CC08091E80083FD3AC078
:103A30008091E80082FD2CC08091E80080FFE9CFF2
:103A40008091F20090E06115710559F08830910580
:103A500040F424912093F100319661507109019650
:103A6000F2CF21E0089709F020E08091E8008E77FE
:103A70008093E800CECF2111CFCF0AC080911904E6
:103A8000882361F0853061F08091E80083FD0AC0F1
:103A90008091E80082FFF2CF80E0089582E00895EF
:103AA00083E0089581E008951F93CF93DF93CDB70E
:103AB000DEB7AA970FB6F894DEBF0FBECDBFEAE11E
:103AC000F4E08091F100819324E0E232F207C9F73B
:103AD0000E9498198091E80083FF2EC180911A04FA
:103AE00090911B04492F50E04A30510508F024C141
:103AF000FA01E95DFE4F0C943032803821F08238B3
:103B000009F01AC108C080911604909117049923F6
:103B100089F082600FC080911E048F70853008F09C
:103B20000BC18093E9008091EB0085FB882780F929
:103B30001092E9009091E800977F9093E8008093BD
:103B4000F1001092F100D1C0282F2D7F09F0F4C0B0
:103B5000882319F0823061F0EFC080911C0481301D
:103B600009F0EAC0933009F080E0809317042EC07A
:103B700080911C0481112AC080911E048F702FEF48
:103B8000280F243008F0D8C08093E9002091EB0082
:103B900020FF1CC0933021F48091EB00806214C0A0
:103BA0009091EB0090619093EB0021E030E0A9014F
:103BB00002C0440F551F8A95E2F74093EA00109225
:103BC000EA008091EB0088608093EB001092E9009E
:103BD0008091E800877F8093E8000E94FC1BACC0C6
:103BE0008111AAC010911C041F778091E300807896
:103BF000812B8093E3008091E800877F8093E80029
:103C00000E94FC1B8091E80080FFFCCF8091E300C4
:103C100080688093E300111102C082E001C083E05C
:103C20008093190489C08058823008F085C0809143
:103C30001C0490911D048C3D53E0950779F583E0B9
:103C40008A838AE289834FB7F894DE01139620E0D5
:103C50003EE051E2E32FF0E050935700E49120FF63
:103C600003C0E295EF703F5FEF708E2F90E0EA3077
:103C700010F0C79601C0C0968D939D932F5F24319D
:103C800049F74FBF8091E800877F8093E8006AE2A0
:103C900070E0CE0101960E949B1C16C060911E042C
:103CA00070911F04AE014F5F5F4F0E945B1BBC0110
:103CB000892B09F441C09091E800977F9093E80028
:103CC00089819A810E94F61C8091E8008B7780930D
:103CD000E80032C0803881F58091E800877F8093CA
:103CE000E800809115048093F1008091E8008E77C0
:103CF00072CF811121C080911C0490911D049927DD
:103D00000297D4F48091E800877F8093E800809147
:103D10001C04809315040E94FC1B809115048111E2
:103D200006C08091E30087FD02C081E001C084E00D
:103D3000809319040E9489198091E80083FF0AC0CA
:103D40008091E800877F8093E8008091EB0080629B
:103D50008093EB00AA960FB6F894DEBF0FBECDBFDE
:103D6000DF91CF911F9108950E94111F0E94141F8F
:103D7000E0EEF0E0808181608083E8EDF0E080811A
:103D80008F77808319BCE3E6F0E0808181608083D7
:103D90001092180408950E94111F0E94141F809110
:103DA000D8008F778093D8008091D8008068809366
:103DB000D8008091D8008F7D8093D80084E089BDA1
:103DC00086E089BD09B400FEFDCF1092190410925F
:103DD0001504109217041092160442E060E080E08F
:103DE0000E94C71B8091E1008E7F8093E10080914B
:103DF000E20081608093E2008091E200886080931D
:103E0000E2008091E0008E7F8093E0000895E3E679
:103E1000F0E080818E7F808381E0809318040C9491
:103E2000CB1E1092E20008951092E10008951F92B7
:103E30000F920FB60F9211242F933F934F935F93DE
:103E40006F937F938F939F93AF93BF93EF93FF9362
:103E50008091E10082FF0BC08091E20082FF07C0E9
:103E60008091E1008B7F8093E1000E94C11F8091CF
:103E7000E10080FF19C08091E20080FF15C08091B1
:103E8000E2008E7F8093E2008091E2008061809367
:103E9000E2008091D80080628093D80019BC85E050
:103EA000809319040E94801A8091E10084FF30C041
:103EB0008091E20084FF2CC084E089BD86E089BD4A
:103EC00009B400FEFDCF8091D8008F7D8093D8008B
:103ED0008091E1008F7E8093E1008091E2008F7EEF
:103EE0008093E2008091E20081608093E200809103
:103EF0001504882311F084E007C08091E30087FD5A
:103F000002C081E001C083E0809319040E94951AE9
:103F10008091E10083FF24C08091E20083FF20C0F4
:103F20008091E100877F8093E10082E08093190413
:103F3000109215048091E1008E7F8093E1008091C2
:103F4000E2008E7F8093E2008091E20080618093A6
:103F5000E20042E060E080E00E94C71B0E948819F6
:103F6000FF91EF91BF91AF919F918F917F916F9151
:103F70005F914F913F912F910F900FBE0F901F9027
:103F800018950895CF93809119048823A1F0C091CA
:103F9000E900CF709091EC00892F817090FD80E84E
:103FA000C82B1092E9008091E80083FD0E94541D07
:103FB000CF70C093E900CF9108959093120380933E
:103FC00011030895E0911103F0911203309721F04D
:103FD0000190F081E02D099480E00895EF92FF9226
:103FE0000F931F93CF93DF93E0911103F09112038E
:103FF0003097B1F18C010280F381E02D0995809119
:10400000070482FF2DC080FF04C083E897E00E9470
:104010009C04E80110E28DE7E82E87E0F82E8091FD
:10402000070480FF0BC088811F928F93FF92EF924D
:104030000E9435050F900F900F900F901150219610
:104040001111EDCF8091070480FF0AC08BE797E044
:10405000DF91CF911F910F91FF90EF900C949C04F2
:10406000DF91CF911F910F91FF90EF9008951F93D3
:10407000CF93DF932091110330911203232BB1F0E2
:10408000EC0118810E94CF309881892B88830E948F
:104090008C0C9881892B8883E0911103F091120395
:1040A0000480F581E02DCE0109951883DF91CF9131
:1040B0001F910895CF93DF9320910F033091100348
:1040C0002817390709F19093100380930F03E091AB
:1040D0001103F09112033097B9F0EC010680F781DB
:1040E000E02D09958091070482FF0EC080FF0CC06F
:1040F000DF93CF938DE697E09F938F930E943505D2
:104100000F900F900F900F90DF91CF910895CF9364
:10411000DF9320910D0330910E032817390709F121
:1041200090930E0380930D03E0911103F09112031D
:104130003097B9F0EC010084F185E02D099580916C
:10414000070482FF0EC080FF0CC0DF93CF938DE584
:1041500097E09F938F930E9435050F900F900F90DB
:104160000F90DF91CF9108950C9475210E94A42D9A
:104170000C94610C8F929F92AF92BF92CF92DF927C
:10418000EF92FF920F931F93CF93DF9300D000D055
:104190001F92CDB7DEB70E94631704E113E0F12C44
:1041A0008F2D0E94680C4C01F801A080B180A826D8
:1041B000B926A114B10439F4F3940E5F1F4FF8E04F
:1041C000FF12EECF39C08091070481FD0E94892142
:1041D000E12CCC24C394D12CC5018C219D21892BA9
:1041E00021F1E982FA8221E0C4018C219D21892BF1
:1041F00009F420E02B830E94AD2D8160782F9D83F0
:104200008C8349815A816B818D810E94BF214981B4
:104210005A816B817C818D810E94442DF8018081BF
:1042200091818C259D2591838083E394CC0CDD1CAA
:10423000F0E1EF12D1CFC0CF8FEF89838A831B8249
:104240000E94AD2D8160782F9D838C8349815A8196
:104250006B818D810E94BF210E94432D0E941D30E1
:104260000E94E21F90911303891759F10E94E21FE7
:10427000809313039091070492FF0EC090FF0CC02F
:104280001F928F938EE897E09F938F930E9435053E
:104290000F900F900F900F90809113030F900F903D
:1042A0000F900F900F90DF91CF911F910F91FF9082
:1042B000EF90DF90CF90BF90AF909F908F900C9435
:1042C000552D0F900F900F900F900F90DF91CF9181
:1042D0001F910F91FF90EF90DF90CF90BF90AF9024
:1042E0009F908F9008950C94A20C0895CF93C62FA1
:1042F0000E94680C21E030E002C0220F331FCA95F3
:10430000E2F72823392381E0232B09F480E0CF91C1
:104310000895EF92FF920F931F93CF93DF9385EA57
:1043200097E00E949C04C0E0D0E080E2E82E81E0AB
:10433000F82E09E917E08C2F0E94680C0E942F2D9F
:10434000FF92EF929F938F93DF93CF931F930F93DF
:104350000E94350521968DB79EB708960FB6F89442
:104360009EBF0FBE8DBFC830D10529F7DF91CF9119
:104370001F910F91FF90EF90089508950895CF93A6
:10438000DF93CDB7DEB72B970FB6F894DEBF0FBE25
:10439000CDBF942F4F83252F588769877A878B87C6
:1043A0004A855B85452B31F02F3F31F481E09F3FFB
:1043B00019F403C081E001C080E080FD07C04F8197
:1043C000588569857A858B850E94442DDE0111967A
:1043D00086E0FD0111928A95E9F785E0FE013796A6
:1043E00001900D928A95E1F749815A816B817C8118
:1043F0008D819E810E9429292B960FB6F894DEBFED
:104400000FBECDBFDF91CF910895882309F4BBC0C3
:104410009CEF980F913A18F40E94132C0DC090E273
:10442000980F983058F4877091E001C0990F8A95E1
:10443000EAF7892F0E94B82C0C94F22C9BE5980F78
:10444000933070F4853A29F0863A31F083E890E0B1
:1044500005C081E890E002C082E890E00C945A2008
:1044600098E5980F973108F08EC0883A09F445C056
:10447000893A09F445C08A3A09F445C08B3A09F4EF
:1044800045C08C3A09F445C08D3A09F445C08E3ACE
:1044900009F445C08F3A09F445C0813B09F445C091
:1044A000803B09F445C0823B09F445C0833B09F4D5
:1044B00045C0843B09F445C0853B09F445C0863BB3
:1044C00009F445C0873B09F445C0883B09F445C061
:1044D000893B09F445C08A3B09F445C08B3B09F48C
:1044E00045C08C3B09F445C08D3B09F445C08E3B6B
:1044F00009F445C080E090E044C082EE90E041C005
:1045000089EE90E03EC08AEE90E03BC085EB90E003
:1045100038C086EB90E035C083EB90E032C084EB8E
:1045200090E02FC087EB90E02CC08CEC90E029C08D
:104530008DEC90E026C083E891E023C08AE891E00A
:1045400020C082E991E01DC084E991E01AC081E2B7
:1045500092E017C083E292E014C084E292E011C0BE
:1045600085E292E00EC086E292E00BC087E292E024
:1045700008C08AE292E005C08FE690E002C080E7C2
:1045800090E00C9487200895882329F19CEF980FE0
:10459000913A18F40E94632C0DC090E2980F983065
:1045A00058F4877091E001C0990F8A95EAF7892F36
:1045B0000E94BE2C0C94F22C9BE5980F933020F4B3
:1045C00080E090E00C945A20885A873120F480E0F3
:1045D00090E00C9487200895882321F00E94B82C45
:1045E0000C94F22C0895882321F00E94BE2C0C9488
:1045F000F22C08950E94D82C0E94A72C0E94F22C25
:104600000E94C3300E94902F80E090E00E945A20C8
:1046100080E090E00C9487200E94C82C0C94FA2231
:10462000CF92DF92EF92FF920F931F93CF93DF937E
:1046300000D000D01F92CDB7DEB76C010E94572D7D
:10464000811118C385E0F601DE01119601900D92EB
:104650008A95E1F7F601408151812381348121154A
:10466000310531F05F3F31F481E04F3F19F403C071
:1046700081E001C080E080FDFDC2F601F280E580AE
:10468000E2948FE0E82249835A83FB82722F3D83B4
:104690002C836F2D8D810E94882B8C010E94872B8B
:1046A0000E94812AE12FE295EF708E2F90E0FC01AD
:1046B000EF5CFE4F0C943032812F807F1F70882377
:1046C00011F01295107FFF20B9F0112329F0812FEE
:1046D0000E94CB2C0E94F22C802F0F900F900F90F5
:1046E0000F900F90DF91CF911F910F91FF90EF905E
:1046F000DF90CF900C940522802F0E94C4221123BA
:1047000009F4B8C2812F0E94D12C0F900F900F9006
:104710000F900F90DF91CF911F910F91FF90EF902D
:10472000DF90CF900C94F22C812F807F1F7080320D
:1047300011F01295107F002319F0013009F12BC000
:10474000FF20A9F0EE2059F1F1E0812FEF1228C0EF
:104750000F900F900F900F900F90DF91CF911F91BE
:104760000F91FF90EF90DF90CF900C94DB2CEE2018
:1047700021F021E0E21609F47DC20E94DE2C4DC03A
:10478000FF20E9F085E08E1508F474C20E94B52C74
:10479000812329F042C0FF20F1F1E11015C0812FE3
:1047A0000F900F900F900F900F90DF91CF911F916E
:1047B0000F91FF90EF90DF90CF900C94EC2294E05B
:1047C0009E1508F457C229C0F601858180FF13C0E9
:1047D0008F708583E4CF003F09F489C108F055C18B
:1047E00080E4800F803208F459C1FF2009F4EAC147
:1047F000EE2009F49AC1802F0E940522093309F0A6
:10480000DAC1FFEF21EE84E0F15020408040E1F773
:1048100000C000002FC2E110D7C1812F59C1812FE4
:1048200086958695837019F08130B9F023C2FF20F8
:1048300019F0C801937002C080E090E00F900F90D3
:104840000F900F900F90DF91CF911F910F91FF90DC
:10485000EF90DF90CF900C945A20FF2019F0C80100
:10486000937002C080E090E00F900F900F900F9037
:104870000F90DF91CF911F910F91FF90EF90DF90FC
:10488000CF900C948720802FFF2019F00E94A32E38
:1048900002C00E940B2F0F900F900F900F900F905F
:1048A000DF91CF911F910F91FF90EF90DF90CF900C
:1048B0000C94902F812F837009F070C0F110DAC131
:1048C000202F229526952770220F220F602F6F70C0
:1048D000862F90E0A0E0B0E06C017D01022E04C0C4
:1048E000CC0CDD1CEE1CFF1C0A94D2F704FF12C096
:1048F0008FE090E0A0E0B0E004C0880F991FAA1FED
:10490000BB1F2A95D2F7BC01CD01609570958095AB
:10491000909503C060E070E0CB011695169513707A
:104920001230B1F040F56C297D298E299F29113074
:1049300031F10F900F900F900F900F90DF91CF916A
:104940001F910F91FF90EF90DF90CF900C949C2AD5
:104950006C297D298E299F290F900F900F900F9021
:104960000F90DF91CF911F910F91FF90EF90DF900B
:10497000CF900C94B62A0E949C2AC701B6010F90D2
:104980000F900F900F900F90DF91CF911F910F918B
:10499000FF90EF90DF90CF900C94822AFF2019F0C7
:1049A000812F817001C08695882309F463C1202F6F
:1049B000229526952770220F220F602F6F70862F69
:1049C00090E0A0E0B0E06C017D01022E04C0CC0CB0
:1049D000DD1CEE1CFF1C0A94D2F704FF12C08FE00E
:1049E00090E0A0E0B0E004C0880F991FAA1FBB1F91
:1049F0002A95D2F7BC01CD01609570958095909570
:104A000003C060E070E0CB0116951695137012306C
:104A1000B1F040F56C297D298E299F29113031F1A3
:104A20000F900F900F900F900F90DF91CF911F91EB
:104A30000F91FF90EF90DF90CF900C94632B6C2937
:104A40007D298E299F290F900F900F900F900F9026
:104A5000DF91CF911F910F91FF90EF90DF90CF905A
:104A60000C94752B0E94632BC701B6010F900F9019
:104A70000F900F900F90DF91CF911F910F91FF90AA
:104A8000EF90DF90CF900C94512B023F09F45EC061
:104A900008F449C0033F09F46CC0A7CE902F907171
:104AA000E92E812F8F71FF2051F00E94EA2A802F7A
:104AB000EE2019F08295807F73CE8F7071CE0E94A8
:104AC0000B2B802FEE2019F08295807F01C08F7014
:104AD0000F900F900F900F900F90DF91CF911F913B
:104AE0000F91FF90EF90DF90CF900C94F322FF2076
:104AF000A9F0E4E0EE1508F4BDC0812F8F710F908E
:104B00000F900F900F900F90DF91CF911F910F9109
:104B1000FF90EF90DF90CF900C94302BF5E0FE15D6
:104B200008F4A8C0EACFFF2099F0812F8F710F9071
:104B30000F900F900F900F90DF91CF911F910F91D9
:104B4000FF90EF90DF90CF900C94EA2AFF2069F35A
:104B5000812F8F710F900F900F900F900F90DF911A
:104B6000CF911F910F91FF90EF90DF90CF900C9419
:104B70000B2BFF2089F0812F8F710F900F900F90DA
:104B80000F900F90DF91CF911F910F91FF90EF90B9
:104B9000DF90CF900C94D52A0F900F900F900F902C
:104BA0000F90DF91CF911F910F91FF90EF90DF90C9
:104BB000CF900C94D02A033509F423CE073409F0A2
:104BC00059C01FCEEE2021F2802F0F900F900F9032
:104BD0000F900F90DF91CF911F910F91FF90EF9069
:104BE000DF90CF900C94C422412F4F70602FC601EC
:104BF0000E94192E0F900F900F900F900F90DF9141
:104C0000CF911F910F91FF90EF90DF90CF900C9478
:104C1000DC2901112FC0FF2069F10E940C232FEF26
:104C200080E792E0215080409040E1F700C0000012
:104C30000F900F900F900F900F90DF91CF911F91D9
:104C40000F91FF90EF90DF90CF900C94FA2D412FB1
:104C50004F70602FC6010F900F900F900F900F9024
:104C6000DF91CF911F910F91FF90EF90DF90CF9048
:104C70000C941C2E0F900F900F900F900F90DF91BF
:104C8000CF911F910F91FF90EF90DF90CF900895FB
:104C90001F93CF93DF9300D000D01F92CDB7DEB724
:104CA000942F4983252F5A836B837C838D834C817A
:104CB0005D81452B31F02F3F31F481E09F3F19F4A6
:104CC00003C081E001C080E0182F117080FD24C076
:104CD00049815A816B817C818D810E94882B292F8B
:104CE00022952F702C3030F42A3048F42250223094
:104CF00068F013C02C3061F02F3051F00EC0803CB2
:104D000028F0803E50F0815F833038F011E005C01C
:104D100093FB112710F901C010E0812F0F900F9025
:104D20000F900F900F90DF91CF911F910895CF9327
:104D3000DF9300D000D01F92CDB7DEB70F900F9059
:104D40000F900F900F90DF91CF910895CF93DF9345
:104D500000D000D000D0CDB7DEB726960FB6F894BD
:104D6000DEBF0FBECDBFDF91CF910895CF93DF930C
:104D7000C091240380912503C817A1F0D0E0CE0193
:104D800066E070E00E940B32FC01EA5DFC4F40815E
:104D9000518162817381848195810E94A62621962A
:104DA000C770E8CFDF91CF9108954091560350919D
:104DB0005703609158037091590380915A03909161
:104DC0005B030C94A6261F93CF93DF9380915B0324
:104DD00082958F7009F05CC080915803882309F494
:104DE00057C02091240310912503C0915603D09100
:104DF0005703A0915903B0915A0381E0CF3F09F0C6
:104E000080E0482F211709F443C0109721F0DF3FBD
:104E100021F080E003C081E001C0842F30E080FDFC
:104E200033C0C90166E070E00E940B32FC01EA5D0C
:104E3000FC4F81818D1328C080818C1325C0828115
:104E4000811122C0838194818A1B9B0B883C910530
:104E5000D8F480915B038F70806180935B03C901FC
:104E600066E070E00E940B32FC01E55DFC4F908132
:104E70009F709061908386E593E00E941023DF91FC
:104E8000CF911F910C94B6262F5F3F4F2770BACF5A
:104E9000DF91CF911F9108959F92AF92BF92CF92D1
:104EA000DF92EF92FF920F931F93CF93DF93CDB7D3
:104EB000DEB761970FB6F894DEBF0FBECDBF8C0191
:104EC00085E0F801DE011D9601900D928A95E1F7CB
:104ED000F80140812181F280C380D48090915603F3
:104EE000309157036091590370915A036115710510
:104EF00031F03F3F31F481E09F3F19F403C081E07E
:104F000001C080E0F82FF1709F2E80FD59C186E529
:104F1000A82E83E0B82EE0905803F601E61BF70BAD
:104F2000EE2009F4EDC080915B03582F507FE83CE0
:104F3000F10508F0A7C0511156C0231313C049133F
:104F400011C0EF2CF1100EC08F70806180935B0355
:104F50000E94D526C5010E94102380915B03F801B1
:104F6000858364C1C114D10431F02F3F31F481E055
:104F70004F3F19F403C081E001C080E080FD03C011
:104F800081E08F2502C080E090E0F82FF170EF2ED5
:104F900080FF1FC0E091240330912503E31709F43B
:104FA00021C1F0E0CF0166E070E00E940B32DC012D
:104FB000AA5DBC4F11968C911197281307C08C9154
:104FC000481304C012968C91F81203C03196E77012
:104FD000E5CFEF2CFF2009F429C180915B038160AC
:104FE00080935B0364C0231306C0491304C0F1100F
:104FF00002C0F801A9C04D872E87FF867C2DD98A73
:10500000C88A522F6F2D89890E9448268823A1F1D2
:10501000FF2091F120915B03822F82958F7090E0A9
:10502000029774F0809156039091570398878F836D
:105030001986DB86CA862C87CE0107960E9410232C
:1050400086E0F801A6E5B3E001900D928A95E1F7BC
:105050000E94E3260E94D52612C0231751F14D87E6
:105060002E87FF867C2DD98AC88A522F6F2D898979
:105070000E94482681112CC0C8010E941023EE24F2
:10508000E394D4C05111E9CF7C2DD98AC88A522F1C
:105090006F2D89890E94972686E593E00E94102350
:1050A00086E0F50111928A95E9F70E94D526E12C58
:1050B000BDC04913D4CFF110D2CFF8018583C80108
:1050C0000E94102386E0F50111928A95E9F7AEC09F
:1050D000FF2091F220915B03822F82958F7090E0E8
:1050E00002970CF4ADCF80915603909157039A83A9
:1050F00089831B82DD82CC822E83CE0101969ECFD6
:10510000E83CF10508F04CC0EF2CFF2009F4B4CFC7
:10511000231330C049132EC020915B0320FD21C012
:10512000822F82958F70482F50E041155105C9F0AC
:10513000F80125834F30510541F08F5F982F9295EC
:10514000907F822F8F70892B8583C8010E94102346
:1051500086E0F801A6E5B3E001900D928A95E1F7AB
:105160002CC086E0F801A6E5B3E001900D928A9587
:10517000E1F75CC04D872E87FF867C2DD98AC88ACF
:10518000522F6F2D89890E944826811159CF809115
:105190005B03816080935B03C8010E94102346C0BB
:1051A0007C2DD98AC88A522F6F2D89890E94972613
:1051B00086E0F50111928A95E9F70E94D52636C05E
:1051C000FF2009F459CF4D872E87FF867C2DD98A81
:1051D000C88A522F6F2D89890E944826882309F496
:1051E0004BCF2ECF7C2DD98AC88A522F6F2D89891B
:1051F0000E94882B292F22952F70223028F49F702F
:1052000039F0811105C00BC0243028F49F7049F497
:10521000805E883020F0C8010E9410239E2CE92C6B
:1052200005C0F8019581907F99F7F9CF8E2D619691
:105230000FB6F894DEBF0FBECDBFDF91CF911F91A7
:105240000F91FF90EF90DF90CF90BF90AF909F9025
:105250000895CF93DF93CDB7DEB72C970FB6F894B0
:10526000DEBF0FBECDBF4F83588769877A878B8794
:105270009C87CE0107960E944C278823D1F09F81FE
:1052800088852A853B85232B31F08F3F31F481E0DF
:105290009F3F19F403C081E001C080E080FD6FC032
:1052A0004F81588569857A858B859C850E94A626C5
:1052B00066C086E0FE013796DE01119601900D92E0
:1052C0008A95E1F7FF81E8856A857B85611571051F
:1052D00031F0EF3F31F481E0FF3F19F403C081E08A
:1052E00001C080E080FD4BC08091250390E09C01CF
:1052F0002F5F3F4F277033274091240350E024173E
:10530000350709F443C0F983EA837D836C8366E043
:1053100070E00E940B32DC01AA5DBC4F96E0FE01FA
:10532000319601900D929A95E1F7209325030E9402
:10533000B62625C090E066E070E00E940B328A5DE0
:105340009C4F0E944C27882371F18091240390E0A8
:1053500066E070E00E940B32FC01EA5DFC4F408188
:10536000518162817381848195810E94A6268091FA
:10537000240390E0019687709927809324038091FD
:105380002403909125038913D5CF0DC00E940C23CF
:105390001092250310922403E6E5F3E086E0DF0196
:1053A0001D928A95E9F72C960FB6F894DEBF0FBED2
:1053B000CDBFDF91CF910895DF92EF92FF920F93CF
:1053C0001F93CF93DF93FC01892B09F488C0E12C54
:1053D000F12CDD24D394EF0121968491853709F4D3
:1053E00060C058F4843708F04EC0843008F068C0BC
:1053F0008130D1F0823071F172C0883709F45BC01E
:1054000050F4863709F453C0873709F068C08E2DF1
:105410000E94C52C52C09CE7980F903708F05FC0DF
:105420008F770E94C4224EC08F010E5F1F4FFE0176
:10543000849190E2980F983050F48770FD2D01C050
:10544000FF0F8A95EAF78F2F0E94CB2C15C00E9480
:10545000052214C08F010E5F1F4FFE01849190E260
:10546000980F983068F48770FD2D01C0FF0F8A9562
:10547000EAF78F2F0E94D12C0E94F22CE80122C063
:105480000E94C422FBCFCF010296FE01C491CC231F
:1054900061F0EFE9FFE03197F1F700C00000C15083
:1054A000F6CFCF010296FE01F490EC010BC00E94F2
:1054B000B52CE82E07C00E94C82C0E94F22C02C016
:1054C0000E9405228F2D882341F0EFE9FFE03197FC
:1054D000F1F700C000008150F6CFFE017CCFDF91D4
:1054E000CF911F910F91FF90EF90DF9008956093FF
:1054F000DC037093DD038093DE039093DF030C9451
:10550000542D08950F931F930091E0031091E10330
:105510002091E2033091E303602B712B822B932BBC
:105520006093E0037093E1038093E2039093E303BD
:105530001F910F910C94532D0F931F930091E00333
:105540001091E1032091E2033091E3036023712382
:10555000822393236093E0037093E1038093E2033B
:105560009093E3031F910F910C94532D0F931F936E
:105570000091E0031091E1032091E2033091E303F5
:1055800060277127822793276093E0037093E103DC
:105590008093E2039093E3031F910F910C94532D9A
:1055A00060E070E0CB010C94772A0F931F9341E0E9
:1055B00050E060E070E08A019B0104C0000F111F01
:1055C000221F331F8A95D2F7C901B8011F910F918D
:1055D0000C94772A0F931F9341E050E060E070E055
:1055E00004C0440F551F661F771F8A95D2F780911C
:1055F000DC039091DD03A091DE03B091DF038A010B
:105600009B01082B192B2A2B3B2BC901B8011F9199
:105610000F910C94772A0F931F9341E050E060E0C4
:1056200070E004C0440F551F661F771F8A95D2F79C
:1056300040955095609570958091DC039091DD03C5
:10564000A091DE03B091DF038A019B010823192397
:105650002A233B23C901B8011F910F910C94772A8B
:105660000F931F9341E050E060E070E004C0440FEE
:10567000551F661F771F8A95D2F78091DC039091A2
:10568000DD03A091DE03B091DF038A019B010827AF
:1056900019272A273B27C901B8011F910F910C94A4
:1056A000772A0F931F930091DC031091DD03209163
:1056B000DE033091DF03602B712B822B932B1F9124
:1056C0000F910C94772A0F931F930091DC03109194
:1056D000DD032091DE033091DF03602371238223F9
:1056E00093231F910F910C94772A0F931F9300918E
:1056F000DC031091DD032091DE033091DF0360278E
:105700007127822793271F910F910C94772A089570
:105710008F929F92AF92BF92DF92EF92FF920F9380
:105720001F93CF93DF9300D000D01F92CDB7DEB789
:105730006B837C838D838A018C819D81892B31F0E1
:105740001F3F31F481E04F3F19F403C081E001C0F5
:1057500080E080FF03C080E090E054C08B8188230C
:1057600009F43DC08090DC039090DD03A090DE033F
:10577000B090DF038091E0039091E103A091E203F8
:10578000B091E303882A992AAA2ABB2A2FE1E22EA4
:10579000F12CD501C4010E2C04C0B695A7959795A0
:1057A00087950A94D2F780FD06C081E0E81AF108D7
:1057B00080F7D12C07C0DE2CB8018E2D0E94730C0F
:1057C000019799F3E12FF0E094E0EE0FFF1F9A9517
:1057D000E1F7E45AFC4FE00FF11DD0820CC0E12F3D
:1057E000F0E084E0EE0FFF1F8A95E1F7E45AFC4FEA
:1057F000E00FF11DD08009831A8369817A818D2D94
:105800000E94730C0F900F900F900F900F90DF91EC
:10581000CF911F910F91FF90EF90DF90BF90AF90CD
:105820009F908F90089590911101992379F1909113
:105830001201992359F1982F9695969596959F3137
:10584000A1F0E0911301F0911401E90FF11D8770AF
:1058500021E030E0A90102C0440F551F8A95E2F70C
:10586000CA019181892B818308959091070490FF4B
:1058700029C01F928F9388ED97E09F938F930E948A
:1058800035050F900F900F900F9008952091130100
:1058900030911401F90132969FEF40E05191851744
:1058A00089F09F3F19F4511101C0942F4F5F4E3181
:1058B000A9F79F3F39F0F901E90FF11D97FDFA951E
:1058C00082830895089590911101992381F1909117
:1058D0001201992361F1982F9695969596959F318F
:1058E000A9F0E0911301F0911401E90FF11D877007
:1058F00021E030E0A90102C0440F551F8A95E2F76C
:10590000CA0180959181892381830895909107042C
:1059100090FF1CC01F928F938AEB97E09F938F9309
:105920000E9435050F900F900F900F900895E09111
:105930001301F09114019F01225E3F4F9281891360
:1059400001C012823196E217F307C1F7089581E092
:1059500090E0E0911301F0911401E80FF91F10821B
:10596000019680329105A9F7089580910604089563
:1059700090910604892B8093060408958095909158
:1059800006048923809306040895809306040895ED
:1059900010920604089590910504892B80930504C4
:1059A00008958095909105048923809305040895B6
:1059B0001092050408958093E40308951092E4037F
:1059C00008958091130190911401FC0131969C017E
:1059D000205E3F4F80E0919191118F5FE217F307B6
:1059E000D1F70895E0911301F0911401809106041C
:1059F0008083E0911301F09114019081809105045E
:105A0000892B80838091E403882361F0E091130166
:105A1000F09114019081892B80830E94E12C8111E7
:105A20001092E40380911301909114010C94EE1FE5
:105A300090937F0180937E0108958295982F9373B0
:105A4000292F220F220F982F9C7C96959695922BAA
:105A5000892F8575880F9A7A9695892B0895CF930B
:105A6000DF93D92F0E941D2DC82F8D2F0E941D2D31
:105A70002C2F30E0322F2227A901482BCA01DF91B9
:105A8000CF91089508950895CF93DF9300D000D06B
:105A90001F92CDB7DEB70F900F900F900F900F9021
:105AA000DF91CF910895089508950C94732180E0BB
:105AB000089583B7817F8C6083BF83B7816083BF84
:105AC0007894889583B78E7F83BF0895CF930E9483
:105AD000BD210E9463170E94BE21C0E08C2F0E944E
:105AE000680C892B29F4CF5FC830C1F780E001C072
:105AF00081E0CF9108950E94710C0C940C231F92A9
:105B00000F920FB60F9211248F939F93AF93BF9371
:105B10008091080490910904A0910A04B0910B04AB
:105B20004196A11DB11D8093080490930904A09390
:105B30000A04B0930B04BF91AF919F918F910F9086
:105B40000FBE0F901F90189582E084BD93E095BD25
:105B50009AEF97BD80936E0008952FB7F8948091C7
:105B6000080490910904A0910A04B0910B042FBF7E
:105B700008952FB7F89460910804709109048091FA
:105B80000A0490910B042FBF08959C014FB7F8941D
:105B90008091080490910904A0910A04B0910B042B
:105BA0004FBF821B930B089578941F920F920FB6EC
:105BB0000F9211248F939F93AF93BF93809108040A
:105BC00090910904A0910A04B0910B040196A11DC3
:105BD000B11D8093080490930904A0930A04B09324
:105BE0000B04BF91AF919F918F910F900FBE0F90BB
:105BF0001F9018950E94B41EF89487E797E790933A
:105C000001088093000887E090EBDC018093220478
:105C100090932304A0932404B09325049CE088E18E
:105C20000FB6F894A895809360000FBE9093600023
:105C3000FFCF80E090E00895089580910E0480FFEA
:105C40000CC08091180190E065E070E00E940B327A
:105C500095958795959587952EC081FF0AC080916F
:105C6000180190E065E070E00E940B3295958795F1
:105C700022C082FF08C08091180190E065E070E0CA
:105C80000E940B3218C020910F042223D9F03091CA
:105C90001701231780F78091180190E065E070E00C
:105CA0000E940B32622F70E00E940B32632F70E073
:105CB0000E941C32CB018038910538F4009739F4EA
:105CC00081E005C085E090E008958FE7089508958C
:105CD00080910E0480FF08C06091160170E07595F8
:105CE00067957595679523C081FF06C06091160181
:105CF00070E0759567951BC082FF04C06091160126
:105D000070E012C060910F046623A9F02091150184
:105D10006217A0F78091160170E090E00E940B32AC
:105D2000622F70E00E941C326038710540F46115EA
:105D3000710519F406C061E070E0862F08958FE7C1
:105D4000089581E00895803F21F40E941D2E8195E1
:105D500004C0813F29F40E941D2E809312040895EF
:105D6000823F21F40E941D2E819504C0833F29F4B7
:105D70000E941D2E809311040895893F19F40E94FA
:105D8000682E05C08A3F31F40E94682E8195809369
:105D9000130408958B3F21F40E94682E819504C05E
:105DA0008C3F29F40E94682E809314040895843F48
:105DB00021F480911004816017C0853F21F4809107
:105DC0001004826011C0863F21F480911004846029
:105DD0000BC0873F21F480911004886005C0883F84
:105DE00031F48091100480618093100408958D3FF8
:105DF00021F480910E0481600BC08E3F21F48091CC
:105E00000E04826005C08F3F29F480910E048460E7
:105E100080930E040895803F39F48091120487FF27
:105E20006CC01092120469C0813F29F48091120461
:105E30001816BCF362C090911104823F29F497FFB9
:105E40005CC01092110459C0833F19F41916CCF3A9
:105E500054C0893F41F48091130418160CF04DC0D2
:105E6000109213044AC08A3F29F48091130487FFDB
:105E700044C0F6CF8B3F39F48091140487FF3DC0B6
:105E8000109214043AC08C3F29F48091140418161F
:105E9000BCF333C0843F21F4809110048E7F17C07F
:105EA000853F21F4809110048D7F11C0863F21F43D
:105EB000809110048B7F0BC0873F21F480911004E8
:105EC000877F05C0883F31F4809110048F7E8093D6
:105ED000100413C08D3F21F480910E048E7F0BC0FF
:105EE0008E3F21F480910E048D7F05C08F3F29F4F1
:105EF00080910E048B7F80930E0480911104811198
:105F00000EC08091120481110AC080911304811186
:105F100006C080911404811102C010920F040895EC
:105F20008091070483FF7EC08DE198E00E949C046D
:105F3000809110041F928F9388E198E09F938F9334
:105F40000E94350586E198E00E949C04809111042E
:105F5000282F082E000C330B3F938F9383E198E09A
:105F60009F938F930E94350581E198E00E949C04E5
:105F700080911204282F082E000C330B3F938F932F
:105F80008EE098E09F938F930E9435058CE098E017
:105F90000E949C0480911304282F082E000C330BC0
:105FA0003F938F9389E098E09F938F930E943505EC
:105FB00087E098E00E949C0480911404282F082E0A
:105FC000000C330B3F938F9384E098E09F938F9363
:105FD0000E94350581E098E00E949C0480910F04A6
:105FE0001F928F938EEF97E09F938F930E943505BA
:105FF0008CEF97E00E949C0480910E041F928F9377
:1060000089EF97E09F938F930E94350586EF97E085
:106010000E949C048DB79EB74C960FB6F8949EBF15
:106020000FBE8DBF80E194E00E9437200E94AD2D0D
:1060300090930D0480930C0408951F93CF93DF93E6
:1060400080910C0490910D040E94C52DFC012091BB
:106050000F04222321F08091190190E007C0809164
:106060001A0190E06AE070E00E940B32E817F9072D
:1060700008F485C080911104C0911204D0911304DA
:1060800010911404811107C0C11175C0D11173C0E2
:10609000111171C074C02F3F19F02F5F20930F04AE
:1060A000181624F40E941D2E80931104809111046F
:1060B00087FF05C00E941D2E8195809311041C1638
:1060C00024F40E941D2E809312048091120487FFF5
:1060D00005C00E941D2E81958093120460911104C9
:1060E000662331F1C0911204CC2311F1062E000C6D
:1060F000770B880B990B0E940A3123E333E343E3C8
:106100005FE30E946E310E94D230609311046C2FC5
:10611000CC0F770B880B990B0E940A3123E333E3F2
:1061200043E35FE30E946E310E94D2306093120419
:106130001D1624F40E94682E80931304809113048A
:1061400087FF05C00E94682E819580931304111665
:1061500024F40E94682E809314048091140487FF15
:1061600005C00E94682E819580931404DF91CF9121
:106170001F910C94902F2F3F09F08FCFA0CFDF916C
:10618000CF911F910895E0E1F4E085E0DF011D92D9
:106190008A95E9F710920F0410920E0408958091E9
:1061A000100408950E94D9306894B1110C9468319C
:1061B00008950E944D3188F09F5798F0B92F992784
:1061C000B751B0F0E1F0660F771F881F991F1AF0E2
:1061D000BA95C9F714C0B13091F00E946731B1E0AF
:1061E00008950C946731672F782F8827B85F39F0AE
:1061F000B93FCCF3869577956795B395D9F73EF47B
:1062000090958095709561957F4F8F4F9F4F089522
:10621000E89409C097FB3EF4909580957095619540
:106220007F4F8F4F9F4F9923A9F0F92F96E9BB27F6
:106230009395F695879577956795B795F111F8CF72
:10624000FAF4BB0F11F460FF1BC06F5F7F4F8F4FDD
:106250009F4F16C0882311F096E911C0772321F0D3
:106260009EE8872F762F05C0662371F096E8862F6B
:1062700070E060E02AF09A95660F771F881FDAF7C2
:10628000880F9695879597F9089557FD9058440F74
:10629000551F59F05F3F71F04795880F97FB991F85
:1062A00061F09F3F79F08795089512161306140642
:1062B000551FF2CF4695F1DF08C0161617061806CF
:1062C000991FF1CF86957105610508940895E894AA
:1062D000BB2766277727CB0197F908950E94803165
:1062E0000C94FA310E94EC3138F00E94F33120F026
:1062F000952311F00C94E3310C94E9310C9468313E
:106300000E94453178F39923C9F35523B9F3950FCA
:1063100050E0551FAA27EE27FF27BB27002408942B
:10632000679520F4E20FF31FB41F0A1E220F331FDC
:10633000441FAA1F6695A9F7779530F4F30FB41F91
:106340000A1E121E08F46395330F441FAA1F221F52
:10635000769599F7879520F4B40F0A1E121E631FD5
:10636000440FAA1F221F331F8695A9F7862F712D70
:10637000602D11249F5750409AF0F1F088234AF085
:10638000EE0FFF1FBB1F661F771F881F91505040E5
:10639000A9F79E3F510580F00C94E3310C946831CD
:1063A0005F3FE4F3983ED4F3869577956795B7956C
:1063B000F795E7959F5FC1F7FE2B880F911D969586
:1063C000879597F9089597F99F6780E870E060E0F6
:1063D00008959FEF80EC089500240A94161617067E
:1063E00018060906089500240A94121613061406C6
:1063F00005060895092E0394000C11F4882352F029
:10640000BB0F40F4BF2B11F460FF04C06F5F7F4FE0
:106410008F4F9F4F08950024552704C0080E591F21
:10642000880F991F009729F076956795B8F3710545
:10643000B9F7802D952F089597FB072E16F4009439
:1064400007D077FD09D00E94363207FC05D03EF414
:10645000909581959F4F0895709561957F4F089510
:10646000EE0FFF1F0590F491E02D0994AA1BBB1BB2
:1064700051E107C0AA1FBB1FA617B70710F0A61B44
:10648000B70B881F991F5A95A9F780959095BC0165
:08649000CD010895F894FFCF3F
:1064980005EB010000FF8F1731180218C617921775
:1064A800010101E5032808140A321E5F5A3135300C
:1064B800005F3F3F3F3F005F415438340041540084
:1064C8005854005445524D494E414C004E4F4E458C
:1064D800004D4F55534500494E54454C4C49004CCE
:1064E8004F474954454348004558504C4F52455230
:1064F8000044454641554C5400397F222407A506DF
:0E65080083062F064806610600080004000204
:106800008800EA44E944E244040005000600070069
:10681000080009000A000B000C000D000E000F001C
:1068200010001100120013001400150016001700CC
:10683000180019001A001B001C001D001E001F007C
:10684000200021002200230024002500260027002C
:10685000280029002A002B002C002D002E002F00DC
:10686000300031003200330034003500360037008C
:10687000380039003A003B003C003D003E003F003C
:1068800040004100420043004400450046004700EC
:10689000480049004A004B004C004D004E004F009C
:1068A000500051005200530054005500560057004C
:1068B000580059005A005B005C005D005E005F00FC
:1068C0006000610062006300640065A185006700EC
:1068D000680069006A006B006C006D006E006F005C
:1068E0007000710072007300890087008A008B00BD
:1068F000E000E100E200E300E400E500E600E7007C
:106900000100010001000100EA4401000100E2442D
:106910000100010001000100460001004A004B0097
:10692000010001004700480001000100E9440100A6
:106930000100010001000100010001003A003B00DC
:106940003C003D003E003F0040004100420043004B
:10695000010035004C0039000100440045005200A0
:1069600049000100010050004F0029004D004E0079
:1069700051000100010001000100010001000100BF
:1069800001000100010001000100010001000100FF
:1069900001000100010001000100010001004D00A3
:1069A0004A004E004B0001000100010001000100FF
:1069B00001000100010001000100010001000100CF
:1069C00001000100010001000100010001000100BF
:1069D00001000100010001000100010001000100AF
:1069E0000100010001000100490001000100010057
:1069F000010001000100010001000100010001008F
:00000001FF
